:1006EA00C9E420C6B520BFA820BDC920B7D120CFF4
:1006FA00B520CDB300BFA8BAC500D3E0B6EE00CE90
:10070A00B0C7B6BFC6BCBC00B6C1BFA8CAA7B0DCDA
:10071A0000202020202020202020202020202020EF
:10072A002000B3F5CABCBBAF002020202020202027
:10073A00202020200025302E3166004143374133E6
:10074A0045373400D4AA000313010A210004FFFF2D
:10075A00FFFFFFFF0A210006FFFFFFFFFFFF0E2337
:10076A000005FFFFFFFFFFFF523020100A2400059B
:10077A00FFFFFFFFFFFF0E250005FFFFFFFFFFFF43
:10078A00020000000E260005FFFFFFFFFFFF020028
:10079A00000002122000000000000000000000001B
:1007AA0000000000002C00000000000018180830AB
:1007BA000000000000002E000000000000001818D1
:1007CA0000000000000000300000001824424242ED
:1007DA00424242241800000031000000107010103C
:1007EA0010101010107C000000320000003C424241
:1007FA000204081020427E000000330000003C4240
:10080A00420418040242423C00000034000000087E
:10081A0008182848487E08081E0000003500000015
:10082A007E40405C62020242423C00000036000008
:10083A00001C2440405C624242423C0000003700F7
:10084A0000007E4444080810101010100000003800
:10085A000000003C4242423C244242423C0000002A
:10086A003900000038444242463A02022438000065
:10087A0000410000001010282828287C4444EE007B
:10088A000000430000003E4282808080808244381B
:10089A0000000045000000FC4248487848484042B1
:1008AA00FC000000CEB008400C40084017FC104085
:1008BA0033FC3040504097FC10441044104410441C
:1008CA00105410481040C7B6010021083FF8000034
:1008DA00244024407E7C248425283C202420245043
:1008EA003C48248E25040200BFC6060878880848BA
:1008FA000848FE0818881C482A48280E48788B8819
:10090A0008080808080808080808BCBC10201020B5
:10091A001020FDFE1020142019FC3108D0881090F8
:10092A00106010601090110E56042000C9E40808E7
:10093A0010083F0821083FFE21083F0821482128C6
:10094A007F28052809081108210845280210C6B57C
:10095A00080008FE4E20484048FCFE8400A408A473
:10096A004AA44AA484A4085010482086C30200005E
:10097A00BFA80100010001FC0100010001007FFE87
:10098A0001000100014001300118010C01080100B9
:10099A000100BDC92108320827C8445057DEF47443
:1009AA0017D4211447D4F21403881A88E4940494BF
:1009BA000AA61144B7D102403FF802483FF8224044
:1009CA003FFE0442084A1FF4681009100910091072
:1009DA0002C00C383010CFB5007C3F8002200420C2
:1009EA0008401F8003200C103FF8108C04A00890C8
:1009FA001088208442840100CDB31040102023FEC9
:100A0A0020404440F888090413FE20947C9000900A
:100A1A0000901D12E112020E0400D3E00100010051
:100A2A000280046008103FFEC10401003FFC01007F
:100A3A00114019301118211045000200B6EE1000BD
:100A4A0008FE7F9051201EFE228254820C9212923E
:100A5A003E92E29222AA22243E4221820000BAC594
:100A6A001FF01010101010101FF00000FFFE0800F9
:100A7A0008001FF0081000100010011000A000402C
:100A8A00D4AA00001FF80000000000007FFE044006
:100A9A000440044004400840084010422042403EBE
:100AAA000000B3F51000080008047EFE04240824A0
:100ABA001224342458249424124410441084111407
:100ACA0012080000CABC1020183010201048FC84FC
:100ADA0025FE2484440044FC288418841484228437
:100AEA0042FC80840000BBAF08800C800888108C10
:100AFA00109830B050E090C0118012801480108499
:100B0A0010841084107C0000CAA7010009000900A3
:100B1A0011001FF82100410001007FFE0100028040
:100B2A00024004200830101C2008B0DC00403E605F
:100B3A00224022802AFE2B882A882A882A50085096
:100B4A001420122023502288410E0204B6C100400C
:100B5A00404033FC204007FE0104E4A822A02220E2
:0E0B6A0027FE20202050288831042206040493
:101BBE00020B02031A6D1A220004FFFFFFFFFFFF44
:101BCE0006000000000000000000000102030405F2
:0B1C4E00EF1FAC0670011E4C70F62268
:0B1B57007C007E00121C157F327E0017
:101B6200AB07AA06EB1BAE0270011A4E60097F9505
:081B72007E00121C4E80ED22E2
:101BDF00AD07AC06C2A5C2A48C80C2A3D2A3EDF5FB
:081BEF0080C2A3D2A3D2A522FB
:101BF700AD07AC06C2A5D2A48C80C2A3D2A3EDF5D3
:081C070080C2A3D2A3D2A522E2
:061C0F007D077C007E0051
:0E1C1500AB05AA04121BDFAF03AE02021BF7E1
:100FE700C2A1C2A67F0A7E00121B62D2A67D087C20
:100FF700307FE37E00121C157D127C007FE77E00A8
:10100700121C157D317C127FEF7E00121C157D00AE
:101017007C017F017E00121C157D007C077F027E0C
:1010270000121C157D307C107F037E00121C15E416
:10103700FDFC7F04FE121C157D077C027F087E00E5
:10104700121C157D007C077F097E00121C15E4FD2C
:10105700FC7F0AFE121C15E4FDFC7F0CFE121C151A
:10106700E4FDFC7F0DFE121C15E4FDFC7F0FFE1254
:101077001C157DF07C007F107E00121C157F11125D
:101087001C0F7D967C007F127E00121C15E4FDFC70
:101097007F13FE121C157FC87E00121B627D907C99
:1010A700147F107E00121C157D277C027F11121BF6
:1010B700597D1D7F12121B577D007C1A7F137E00FE
:1010C700121C157D337C007F297E00121C157D0EB6
:1010D7007F2B121B57E4FDFC7F20FE121C15E4FD3D
:1010E700FC7F21FE121C157F30121C0F7D067C022F
:1010F7007F317E00121C157D067C057F327E001233
:101107001C157D047C077F357E00121C157D037C32
:10111700127F367E00121C157D077C007F377E000C
:10112700121C15E4FDFC7F38FE121C157D067C079A
:101137007F397E00121C157D017C077F3C7E0012E3
:101147001C157D0F7C007F3D7E00121C15E4FDFC05
:101157007F50FE121C157DEF7C007F517E00121C14
:1011670015E4FDFC7F52FE121C157D3F7C017F5369
:101177007E00121C157D007CA77F607E00121C1567
:101187007D017C007F617E00121C15E4FDFC7F6AF7
:10119700FE121C157D107C007F907E00121C157DB1
:1011A700007C067F927E00121C157D037C007F93D6
:1011B7007E00121C157D107C017F957E00121C1588
:1011C700E4FDFC7F97FE121C15E4FDFC7F98FE12E0
:1011D7001C157D337C017F077E00121C157F647E02
:1011E70000121B62D2A17508FF7509E0750DF8752D
:0311F7000E0022C5
:101B9D008D828C83AD07AC067F207E00121C15ADA7
:101BAD0082AC837F217E00121C157F227E00021BDA
:011BBD00DF48
:101A30008E478F488A4B8B4C8D828C83AD48AC4748
:101A40007F507E00121C15AD4CAC4B7F517E0012B6
:101A50001C15AD82AC837F527E00121C15AD4EACBE
:101A60004D7F537E00121C15AD82AC83AF48AE474C
:031A7000021B9DB9
:10197600752B00752CE774FFF52DF52E7DC87BE6DB
:081986007A007F787C007E00EE
:0C198E008E258F268C278D288A298B2A15
:10199A00852B4D852C4E121A30AB28AA27D3EB95EE
:1019AA002CEA952B5022852682852583D3E58295BC
:1019BA002AE5839529500AAF2EAE2D121BF7A38074
:0819CA00EB0BBB00010A80D504
:0119D20022F2
:041A73008E258F2607
:101A7700754D01754E3F7BEF7A00E4FDFCFFFE12CA
:101A87001A30E4FDFCFFFE121B9DE4FBFA900000F8
:101A9700AF26AE25121BF7A3E582B440F3E583B466
:0D1AA70001EE0BBB00010AEB64F04A70E099
:011AB400220F
:081576008E318F328C338D346D
:10157E00E4F53DF53EF53FF540F541F542F5437591
:10158E004410F53DF53E1205F0FF90079E75F011E3
:10159E00E53E1206A8E53D75F011A42583F583E41A
:1015AE00936F600E053EE53E7002053D6410453DAD
:1015BE0070D4C3E53E9544E53D954340030216883D
:1015CE00E5322407FBE43531FAE534240FF54EE419
:1015DE003533F54DAD34AC33AF32AE31121A30E493
:1015EE00F53FF54090079F75F011E53E1206A8E510
:1015FE003D75F011A42583F583E5822540F582E53E
:10160E0083353FF583E493F9E4F541F54274807E2A
:10161E0000A842088006CEA2E713CE13D8F8FFE941
:10162E00FDEF5D6006AE38AF398008E53C7009AE5F
:10163E003AAF3B121BF7801DE5322542CFE531351F
:10164E0041CF2401CF3400FEE5342540FDE533358E
:10165E003FFC121B9D0542E54270020541C39408F2
:10166E00E541940040A70540E5407002053FC39454
:0A167E0010E53F940050030215F23E
:01168800223F
:081408008E318F328C338D34DC
:10141000E4F53DF53EF53FF540F541F542F54575FE
:101420004615F53DF53E1205F0FF9008AE75F02229
:10143000E53E1206A8E53D75F022A42583F583E478
:1014400093B50721900001120609FF9008AF75F0CF
:1014500022E53E1206A8E53D75F022A42583F5831A
:10146000E4936F600E053EE53E7002053D64154550
:101470003D70B3C3E53E9546E53D954540030215F5
:1014800075E532240FFBE43531FAE534240FF54ECF
:10149000E43533F54DAD34AC33AF32AE31121A30E2
:1014A000E4F53FF540E54025E0FFE53F33FE9008D9
:1014B000B075F022E53E1206A8E53D75F022A425A0
:1014C00083F583E5822FF582E5833EF583E493FC83
:1014D000E54025E0FFE53F33FE9008B175F022E5D9
:1014E0003E1206A8E53D75F022A42583F583E5822A
:1014F0002FF582E5833EF583E493FFECF543EFF5AA
:1015000044E4F541F542E47E80A842088005CEC35C
:1015100013CE13D8F9FFE5435EFEE5445F4E600647
:10152000AE38AF398008E53C7009AE3AAF3B121BCC
:10153000F7801DE5322542CFE5313541CF2401CF7B
:101540003400FEE5342540FDE533353FFC121B9D9C
:101550000542E54270020541C39410E54194004004
:10156000A50540E5407002053FC39410E53F940097
:0515700050030214A568
:011575002253
:101851007BFF752C00752D1F752E07752FE0E4F5A4
:07186100307D96FC7F2DFE97
:101868008E258F268C278D288B298A2A892BAB29B0
:10187800AA2AA92B1205F0FF6067EFD394804029AC
:10188800852C38852D39852E3A852F3B85303CAD02
:1018980028AC27AF26AE2512140874102526F52685
:1018A800E43525F5257402802DAB29AA2AA92B85B4
:1018B8002C38852D39852E3A852F3B85303CAD282F
:1018C800AC27AF26AE2512157674082526F526E432
:1018D8003525F5257401252BF52BE4352AF52A80C5
:0218E8008D224F
:10168900752B00752C45752D00752E1F7BEF7A0083
:10169900E4FDFCFFFE12198E752B00752C5D752D6E
:1016A900F8752E007BEF7A007D467C00E4FFFE1280
:1016B900198E7BFF7A0679EAE4F52CF52D752EF85B
:1016C900F52FF5307D4AFC7F26FE121868752B012F
:1016D900752C3F752D07752EE07BEF7A007D5E7CBA
:1016E90000E4FFFE12198E752B00752CDB752D0099
:1016F900752E1F7B407A007DAA7F0F12198A121955
:1017090076752B01752C0B74FFF52DF52E7DEC12DA
:1017190019847BFF7A0679FFE4F52CF52D752E07E0
:10172900752FE0F5307DD0FC7F50FE1218687BFFE5
:101739007A077904E4F52CF52D752E07752FE0F558
:10174900307DF4FC7F50FE121868752B01752C3C16
:10175900752D00752E1F7BEF7A007D297C017F781E
:101769007E0012198E7BFF7A077909E4F52CF52D95
:10177900752E07752FE0F5307D2B7C017F32FE0237
:021789001868DE
:041C23007F0A7E00B6
:0C1C2700EF4E6007EF1F70F81E80F522E2
:041AE2007FF47E010E
:101AE60075CBFC75CA6975CDFC75CC69C2AD75C878
:101AF60004EF1FAC0670011E4C600730CFFDC2CF4D
:051B060080EFC2CA22BD
:101AB50075CBDC75CA0075CDDC75CC00C2AD75C8BB
:101AC50004EF1FAC0670011E4C600F20CF08300AD2
:0D1AD500FAC2CAC2CF22C2CF80E7C2CA2225
:101B7A007D08AC051DEC6016EE2EFEC295EF339281
:101B8A0097EF2FFFA296E4334206D29580E4D295CE
:021B9A00AF0694
:011B9C002226
:0E1C3300C2937FAA121B7A7FFF121B7AD293F4
:011C41002280
:0D178B007F647E00121AE67B007A00794F21
:061798008B258A2689273B
:10179E00E4F529F528121C33BFF0037528FD121C41
:1017AE00230528E528C3946440EBE52864FE600316
:1017BE0002184EC2937FBB121B7A8F28AB25AA2626
:1017CE00A9277401120636E4F528AB25AA26A92707
:1017DE001205F0FFE528C39F50317FFF121B7AAB35
:1017EE0025AA26A927852882758300EF120648852B
:1017FE00288275830012060962291205F0D39420FF
:10180E004005D2937F0122052880BF121C237FFF43
:10181E00121B7AAB25AA26A927852882758300EF8D
:10182E00120648121C23D293AB25AA26A927852877
:10183E0082758300120609B529037F00227F0122DB
:02184E007F0118
:011850002275
:1019D30078777C007D007B007A0079CC7E007F04E1
:0F19E3001205CA7B007A00796D8B228A23892432
:0619F2008B258A268927DF
:1019F800E4F529C2937FCC121B7AE4F528AB25AA1B
:101A080026A9271205F0FEE528C39E5013852882D3
:101A1800758300120609FF6229121B7A052880DDEA
:071A2800AF29121B7AD293D3
:011A2F002294
:0C1C4200C2927F327E00121AB5D29222AC
:1011FA00E478CAF608F60812068F43528000121BDA
:10120A0032121C42121AE2120FE7E4FFFE121A739C
:10121A001216892094FD1219D312178B78C9A607C2
:10122A00AB22AA23A924900001120609FF7850E6EE
:10123A00B5070578C9E660131219E612178B78C943
:10124A00A6077F647E00121AE680D578CBE6640191
:10125A00184670030214072094FD7F467E00121A76
:10126A00E62094E77522FF7523077524547BFF7ADD
:10127A000779541219F212178B78C9A607AB22AA5A
:10128A0023A924900001120609FF7850E6B5070544
:10129A0078C9E660297BFF7A07799C1219F278C926
:1012AA00A6077A077912121851121AE27BFF7A07F7
:1012BA00791B752C07752DE012185902126B78CC20
:1012CA007C007D007B007A0079517E007F04120544
:1012DA00CA78CC12066AE4FBFA79C078BF12000A0F
:1012EA0078CC120683E4FFFEFDFC78CC1206761257
:1012FA0000FB50307BFF7A07799C1219F278C9A655
:10130A00077A07792C121851121AE27BFF7A0779A9
:10131A0033752C07752DE012185978CA76000876AD
:10132A00010212551219D312178B78C9A607AB22DC
:10133A00AA23A924900001120609FF7850E6B507EE
:10134A000578C9E660131219E612178B78C9A60741
:10135A007F647E00121AE680D57528FF7529077505
:10136A002A3F78CC12066A8F2E8E2D8D2C8C2B7BE1
:10137A00007A0079A9120BD47BFF7A07799C12199B
:10138A00F27BFF7A077945E4F52CF52D74FFF52EEB
:10139A00F52FE4F5307DD0FC7F7DFE1218687B00C6
:1013AA007A0079A9E4F52CF52D74FFF52EF52FE4D2
:1013BA00F5307DF4FC7F7DFE1218687BFF7A077991
:1013CA004EE4F52CF52D74FFF52EF52FE4F5307D5E
:1013DA00F4FC7FB4FE1218687FD07E07121AE61258
:1013EA001976752B01752C0B74FFF52DF52E7BE6FE
:0D13FA007A007DEC12198812197602126B30
:0114070022C2
:101B3200C2AD75C804758780759870758921758DD9
:101B4200FD858D8BD28EC2ABD2AFC2A8D288C2CA5B
:051B5200D2ACC20A2222
:1000030002019DE86480F8E933E83360110460F08D
:10001300ED33EC337009E8FCE9FDEAFEEBFF220463
:1000230060DED3EB9FEA9EE99DE8C2E78CF0C2F75E
:1000330095F0400CE8CCF8E9CDF9EACEFAEBCFFB2A
:1000430012016885D0F05804700320D5B3E804701A
:10005300075002B2D50201A792D5EC0460F7E4CCB5
:10006300C0E0C398F8603B94186008400DD0E0FBF3
:1000730002017FE4FBFAC9FC8028E830E406E4C906
:10008300FBE4CAFCE830E305E4C9CACBFCE8540747
:100093006010F8C3E913F9EA13FAEB13FBEC13FC52
:1000A300D8F130F52FC3E49CFCEF9BFFEE9AFEEDF5
:1000B30099FDD0E0FBEF4E4D4C701222DB030201A1
:1000C300A4EC2CFCEF33FFEE33FEED33FDED30E714
:1000D300EB02017FEF2BFFEE3AFEED39FDD0E0FBA3
:1000E30050130BBB00030201A7ED13FDEE13FEEF4C
:0800F30013FFEC13FC02017F76
:1000FB0074F8CC6480CCC86480C8F582046043C3B8
:10010B00EB9FF5F0EA9E42F0E99D42F0E89C45F04A
:10011B0060305018E5825FFFE582F42B5582FB506F
:10012B00210ABA001D09B90019088016E5825BFB8C
:10013B00E582F42F5582FF50090EBE00050DBD0060
:10014B00010CC3EB9FF5F0EA9E42F0E99D42F0E80B
:0D015B009C45F06007CC4820E701B3EC2282
:100B7800E53C2428F8E6053C227825300702782849
:100B8800E475F0011206B40205F02000EB7F2ED2C6
:100B9800008018EF540F2490D43440D4FF30040B55
:100BA800EF24BFB41A0050032461FFE53D6002152D
:100BB8003D0540E5407002053F30070D7825E47596
:100BC800F0011206B4EF020636021B0B7403D207BB
:100BD8008003E4C207F53C8B258A268927E4F53D86
:100BE800F53FF540E53D60077F20120BB380F575B2
:100BF8003EFFC201C200C202C203C205C206C20849
:100C0800120B81FF700D3007057F00120BC4AF4037
:100C1800AE3F22B4255FC2D5C204120B81FF24D097
:100C2800B40A00501A75F00A783D30D50508B6FFA9
:100C38000106C6A426F620D5047002D20380D92462
:100C4800CFB41A00EF5004C2E5D204020EB1D201AB
:100C580080C6D20080C0D20280BCD2D580BAD2056C
:100C680080B47F20120BB32002077401B53D004009
:100C7800F1120B78FF120BB3020BECD208D20680EC
:100C880095120B78FB120B78FA120B78F94A4B7015
:100C98000679A87A0F7BFF20022EE53D602A7E00A8
:100CA8008E8275830012060960060EEE653E70F0AE
:100CB800C2D5EBC0E0EAC0E0E9C0E0EE120F11D007
:100CC800E0F9D0E0FAD0E0FB1205F0FF60AAEBC033
:100CD800E0EAC0E0E9C0E0120BB3D0E02401F9D0AB
:100CE800E03400FAD0E0FBE53E0460DCD53ED98074
:100CF80087D20280A2120EF460F7E53E700104125A
:100D080001B2A93E600DE53E600914F53E120F9B45
:100D1800EF60F3EA30E702F404C3995077EAF42568
:100D28003E0430E701E404F53E800D120EF460C184
:100D3800EA053E253E1201B2EA783BF630E701E4C7
:100D4800253E04D53E0420050114120F11E4C0E02D
:100D5800120F9B783BE6601320E70714F6120B9BF3
:100D6800802204F6D0E014C0E07F00120B9BE53E21
:100D78006007120B92153E800B300503120B92D0C0
:100D8800E0020BECD0E00480C5120EF460A0E53E52
:100D9800041201B2783BEAF6E53E20050260010440
:050DA8002404120F11EC
:100DAD0074FF04C0E0120F9B120B9BE53E20050261
:100DBD006003120B92D0E0B53EE87F45120BA5788B
:100DCD003BE67F2B30E7047F2DF404C0E0120BB31C
:100DDD00D0E075F00A84C0F0120B9CD0E0120B9C91
:100DED00020BEC791080027908C206C2088008D285
:100DFD00D5790A8004790AC2D5E53E047002F53E24
:100E0D00E4FAFDFEFF120B78FC7B08200113120B98
:100E1D0078FD7B1030000A120B78FE120B78FF7BE9
:100E2D0020EC3382D592D55013C3E43000069FFFDA
:100E3D00E49EFEE42001039DFDE49CFCE4CBF8C29E
:100E4D0001EC700CCFCECDCCE824F8F870F3801700
:100E5D00C3EF33FFEE33FEED33FDEC33FCEB33FB31
:100E6D00994002FB0FD8E9EB300105F8D0E0C448FA
:100E7D00B201C0E00AEC4D4E4F78207B0070C2EA03
:100E8D00B53E0040BCC0E0120F13D0F0D0E0200101
:100E9D0004C4C0E0C4B201C0F0120B9CD0F0D5F078
:100EAD00EB020BEC1206C40C89530DF0580C5A4C86
:100EBD000C56420DF44F0DFC440DFC490C6F430EC6
:100ECD0002550D33460D91450CFD470FC8500C5E74
:100EDD002D0C622E0C852B0C66230C83200FB12A52
:100EED000C1E4800000C7DE53EB4FF03753E061256
:100EFD000B78FC120B78FD120B78FE120B78FF7835
:100F0D00340201E1790AA2D5200314300509B91084
:100F1D00020404B9080104A2D520060250010420E0
:100F2D0002689202B53D005034C0E07F20300319B5
:100F3D007F30A20272067205500F120F6AC202C2F2
:100F4D0006C205C2087F30800F300503E9C0E012EC
:100F5D000BB3300503D0E0F9D0E0B53DCC3005172B
:100F6D007F30B9100C120BB37F583004077F788097
:100F7D0003B90803120BB33002057F2D020BB37FAB
:100F8D00202008F87F2B2006F322920280CF7F00CD
:100F9D00B4070050052434F8E6FF22286E756C6CFA
:100FAD002900D201120B783001F8C201783D30D5FD
:100FBD000108F6020C1E2D50434958120B782403DC
:100FCD00B405004001E4900FC393120BA4743A12C0
:0A0FDD000BA4D203753D04020DF0D1
:10016800E9D2E7C933E833F892D5EDD2E7CD33ECDD
:0701780033FC5002B2D52256
:10017F00EC30E7100FBF000C0EBE00080DBD0004E1
:10018F000BEB6014A2D5EB13FCED92E7FD2274FF8D
:10019F00FCFDFEFF22E480F8A2D574FF13FC7D80E6
:0301AF00E480EFFA
:1001B200F920E72824F950037907E4F42402FB1814
:1001C200DBFDE624FB5014E9600DE4F618E604F6C4
:0F01D200B40A08E4F6D9F57401F60A22C2D52260
:1001E100ED33EC3392D5FA602AB4FF33EDC2E77BED
:1001F100FF60067A027906E4227A02790F20D5049B
:100201007A02790A224E614E002B494E46002D4951
:100211004E4600E47A08F608DAFC7B00740722E80F
:10022100C0E0ECC0E0EDC0E0EEC0E0EFC0E0EA7598
:10023100F010A4CAABF075F04DA42BFBE435F0FC33
:10024100EA2410FAEB34C5FBEC34D9FCEDC2E7FF2C
:1002510075F056A4F42411C5F0F434C58FF0A42A26
:10026100E5F03BE43CF620E7141204BAD0E0FFD0FD
:10027100E0FED0E0FDD0E0FC1203ED8014F40412A6
:1002810004BAD0E0FFD0E0FED0E0FDD0E0FC1202E5
:10029100E4D0E0F8E6FAEDD2E7CD33EC332482FB8B
:1002A100E4C3CF33CFCE33CECD33CD33DBF37B07B6
:1002B10075F00A846004F6081B0AE5F0F6088FF071
:1002C100740AA4FFACF08EF0740AA42CFEACF050BA
:1002D100010C8DF0740AA42CFDE435F0F608DBDE88
:0302E1007407227D
:1002E400EC4D6011E8497017ED33EC3304600DE414
:1002F400FCFFFEFD22E933E8330470F802019D128D
:10030400016858046009E4CC24815006285009028D
:1003140001A72840030201A4C0E0EB4A7044B9805D
:1003240006D0E0FB020193EF4E701CBD8008EBFF8A
:10033400EAFEE9FD80EBE98DF0A4FEE5F00203CDD1
:10034400E9CDF9EAFEEBFFEF89F0A4FCE5F0CE89F4
:10035400F0A42EFFE435F0CD89F0A42DFEE435F0B1
:100364008067EF4E7005BD80D780C3EF8BF0A4ACDF
:10037400F0EE8BF0A42CFCE435F0F8EF8AF0A42C1A
:10038400E5F038FCE433CB8DF0A42CFCE5F03BF82D
:10039400EE8AF0A42CFCE5F038F8E433CF89F0A41D
:1003A4002CFCE5F038CF3400CE89F0A42FFFE5F023
:1003B4003EFEE433C98DF0A42EFEE5F039CD8AF07B
:1003C400A42FFFE5F03EFEE43DFD33D0E0FB5007F3
:1003D4000BBB000F0201A7EC2CFCEF33FFEE33FE46
:0603E400ED33FD02017F74
:1003EA000201A7EC5D046005E85904700302019D4F
:1003FA00120168580460F6EC4860F2EC7004FDFEE5
:10040A00FF22C860DB2481C85009C39860025006E5
:10041A000201A49850CAF582E9294B4A7005AB82B9
:10042A0002019375F0007C1A7880C3EF9BEE9AED77
:10043A0099400DC3EF9BFFEE9AFEED99FDE842F05D
:10044A00DC23ACF0D0E0FFD0E0FED0E0FDAB8220B0
:10045A00E7101BEB60BAEC2CFCEF33FFEE33FEED3A
:10046A0033FD02017FE803F830E705C0F075F000BC
:10047A00EF2FFFEE33FEED33FD40B830E7C280AA1E
:10048A003F8000004120000042C80000447A00007A
:10049A00461C400047C35000497424004B189680FC
:1004AA004CBEBC205A0E1BCA6753C21C749DC5AEF3
:1004BA00FB60065407601C23231204E8EB543860DF
:1004CA00091204D41204E31202E4ECF8EDF9EEFA8C
:1004DA00EFCB22EB1204E380F1543803241C90047E
:1004EA008AFE93FC0EEE93FD0EEE930ECE93FF2240
:030000000218EAF9
:0C18EA00787FE4F6D8FD7581CF0219313B
:1004FA00E709F608DFFA8046E709F208DFFA803EE4
:10050A0088828C83E709F0A3DFFA8032E309F608D0
:10051A00DFFA8078E309F208DFFA807088828C8338
:10052A00E309F0A3DFFA806489828A83E0A3F608EC
:10053A00DFFA805889828A83E0A3F208DFFA804CC6
:10054A0080D280FA80C680D4806980F2803380109D
:10055A0080A680EA809A80A880DA80E280CA803306
:10056A0089828A83ECFAE493A3C8C582C8CCC5837E
:10057A00CCF0A3C8C582C8CCC583CCDFE9DEE7804E
:10058A000D89828A83E493A3F608DFF9ECFAA9F0CD
:10059A00EDFB2289828A83ECFAE0A3C8C582C8CC23
:1005AA00C583CCF0A3C8C582C8CCC583CCDFEADE3C
:1005BA00E880DB89828A83E493A3F208DFF980CC9E
:1005CA0088F0EF60010E4E60C388F0ED2402B40497
:1005DA000050B9F582EB2402B4040050AF2323453E
:0605EA00822390054A7314
:1005F000BB010689828A83E0225002E722BBFE0209
:09060000E32289828A83E493223B
:10060900BB010CE58229F582E5833AF583E02250A6
:1006190006E92582F8E622BBFE06E92582F8E222F0
:0D062900E58229F582E5833AF583E493220A
:10063600BB010689828A83F0225002F722BBFE01A3
:02064600F3229D
:10064800F8BB010DE58229F582E5833AF583E8F0E8
:10065800225006E92582C8F622BBFE05E92582C894
:02066800F2227C
:0C066A00E6FC08E6FD08E6FE08E6FF22BC
:0D067600E6FB08E6F908E6FA08E6CBF822F4
:0C068300ECF608EDF608EEF608EFF622A3
:10068F00D083D082E493F608740193F60874029332
:09069F00F608740393F674047369
:0C06A800A42582F582E5F03583F583225D
:1006B400FAE6FB0808E6F925F0F618E6CA3AF62247
:1006C400D083D082F8E4937012740193700DA3A3C5
:1006D40093F8740193F5828883E4737402936860D9
:0606E400EFA3A3A380DFD9
:101B0B00EFB40A07740D121B16740A309811A899BA
:101B1B00B8130CC2983098FDA899C298B811F6303A
:071B2B0099FDC299F5992212
:1018F6000211FAE493A3F8E493A34003F68001F2FD
:1019060008DFF48029E493A3F85407240CC8C333F2
:10191600C4540F4420C8834004F456800146F6DFC1
:10192600E4800B0102040810204080901BBEE47E78
:10193600019360BCA3FF543F30E509541FFEE493B6
:10194600A360010ECF54C025E060A840B8E493A37D
:10195600FAE493A3F8E493A3C8C582C8CAC583CAA8
:10196600F0A3C8C582C8CAC583CADFE9DEE780BE60
:011BDE000006
:00000001FF
